S02B00002F686F6D652F766F6F72627572672F446576656C6F706D656E742F4F70656E424C542F5461726765E0
S3150800200000800020992D0008E92D0008E92D000818
S3150800201000000000000000000000000000000000B2
S31508002020000000000000000000000000E92D000884
S315080020300000000000000000E92D0008512E0008ED
S31508002040E92D0008E92D0008E92D0008E92D00080A
S31508002050E92D0008E92D0008E92D0008E92D0008FA
S31508002060E92D0008E92D0008E92D0008E92D0008EA
S31508002070E92D0008E92D0008E92D0008E92D0008DA
S31508002080E92D0008E92D0008E92D0008E92D0008CA
S31508002090E92D0008E92D0008E92D0008E92D0008BA
S315080020A0E92D0008E92D0008E92D0008E92D0008AA
S315080020B0E92D0008E92D0008E92D000800000000B8
S309080020C0EE11AA5510
S315080020C410B5064C2378002B07D1054B002B02D0FC
S315080020D4044800E000BF0123237010BDD40000208B
S315080020E400000000A82E0008044B10B5002B03D0EE
S315080020F40349044800E000BF10BDC04600000000C4
S31508002104D8000020A82E0008002243088B4274D366
S3150800211403098B425FD3030A8B4244D3030B8B42D6
S3150800212428D3030C8B420DD3FF22090212BA030CDF
S315080021348B4202D31212090265D0030B8B4219D3C0
S3150800214400E0090AC30B8B4201D3CB03C01A5241E0
S31508002154830B8B4201D38B03C01A5241430B8B4228
S3150800216401D34B03C01A5241030B8B4201D30B0311
S31508002174C01A5241C30A8B4201D3CB02C01A524138
S31508002184830A8B4201D38B02C01A5241430A8B42FB
S3150800219401D34B02C01A5241030A8B4201D30B02E4
S315080021A4C01A5241CDD2C3098B4201D3CB01C01AFE
S315080021B4524183098B4201D38B01C01A5241430908
S315080021C48B4201D34B01C01A524103098B4201D3F6
S315080021D40B01C01A5241C3088B4201D3CB00C01A63
S315080021E4524183088B4201D38B00C01A52414308DB
S315080021F48B4201D34B00C01A5241411A00D2014600
S31508002204524110467047FFE701B5002000F006F872
S3150800221402BDC0460029F7D076E770477047C04626
S3150800222470B588B08024A4020121200000F0A0FC27
S315080022340121200000F08EFC9025ED0501220221E3
S31508002244280000F07BFB01220321280000F076FB1E
S3150800225406A90C26069603234B71013B0B71002431
S315080022648C71013BCB71280000F022FBE1231B0291
S31508002274009301940294039405940496054C6946C4
S31508002284200000F091FC0121200000F0F9FC08B0C0
S3150800229470BDC04600440040F0B5D6464F4680B5EA
S315080022A48DB081468A46019202A800F059FB049B28
S315080022B40093002501E00135EDB2112D1FD8134B0B
S315080022C46A00D65C9B185F78F41901344B465C4364
S315080022D421000098FFF79EFF0029ECD12100009801
S315080022E4FFF712FF80B253461880013880B2084BB4
S315080022F49842E0D8019B1E705F70012000E0002020
S315080023040DB00CBC91469A46F0BDC046C42E0008D2
S31508002314FF030000F0B58BB06B469E1C0123338087
S315080023242C4B1B886A46138001218020800400F008
S315080023341FFC01218020C00200F00CFC264D04225B
S315080023440821280000F0FAFA04220921280000F0DE
S31508002354F5FA08A9C0239B00089302230B710133DD
S315080023644B7100248C7101270123CB71280000F0DE
S315080023749FFA6A4631001948FFF78EFF184800F09D
S3150800238419F905AD280000F027FAAC71EC712C7226
S315080023946C72AC72EC72AC70EC706B461B78013BD9
S315080023A42B716B465B78013B6B7133882B80290054
S315080023B40B4800F00BF901A88472C47207730480F1
S315080023C444808480C4800481477300F083F90BB089
S315080023D4F0BDC046C02E00080004004820A107002E
S315080023E40064004010B504002021064800F058FC9B
S315080023F4012801D0002010BD024800F04DFC2070D1
S315080024040120F8E70044004010B5FFF709FFFFF77D
S3150800241481FF10BDBFF34F8F024A034BDA60BFF347
S315080024244F8FFEE70400FA0500ED00E010B5214BD6
S315080024341B78002B14D12048FFF7D4FF012800D0BD
S3150800244410BD1D4B1B78002BFAD000F0F9FC1B4B72
S3150800245418600122174B1A700022194B1A70EFE7FD
S31508002464174B1B7801331448C018FFF7BBFF012824
S315080024740AD000F0E5FC114B1B6864339842DFD997
S3150800248400220C4B1A70DBE70D4A13780133DBB2D2
S315080024941370094A12789342D2D10022054B1A7056
S315080024A4054B5B78FF2BCBD1034B9B78002BC7D10D
S315080024B4FFF7B0FF31010020F000002034010020AE
S315080024C43201002010B586B00021124800F0E2F966
S315080024D4002801D106B010BD01AC220000210D4828
S315080024E400F08AF9237A002B05D10B4B019A9A42FC
S315080024F40ED0002300E00023012BEBD101ABDB7ADD
S31508002504FF2BE7D101AB1B7B002BE3D1FFF782FF3F
S315080025140123F1E7006400406706000010B5FFF7E1
S3150800252485FFFFF7CFFF10BD10B582B001218020CB
S31508002534800200F00FFB202300931F3B6A461371A9
S3150800254400239371032269464A71CB719024E405EA
S31508002554200000F0ADF92021200000F0EDF902B0CA
S3150800256410BD000010B500F06BFC04000F4B1B688F
S31508002574C31AF422FF3293420ED90D4B1B78002B53
S315080025840BD1F33AFF3A0A4B1A7020219020C00562
S3150800259400F0D0F9054B1C6010BD0022044B1A70DC
S315080025A420219020C00500F0C7F9F3E73C0100207C
S315080025B43801002010B58024A4040121200000F06D
S315080025C4E5FA0021200000F0E1FA10BD03680222B2
S315080025D4934303600368013A13430360002300E04E
S315080025E401334268D20702D4394A9342F8D1436880
S315080025F4DB076AD58B79012B3BD00368802293438A
S315080026040360CB79012B39D00368402293430360D6
S315080026140B7A012B37D003682022934303604B7A45
S31508002624012B35D003681022934303608B7A012B60
S3150800263433D00368082293430360CB7A012B31D045
S3150800264403680422934303608B789B07CA781206AF
S3150800265413430A79120413434A79120513430A8861
S31508002664013A1343C36103680122934303600023B9
S315080026741EE00368802213430360C2E7036840220E
S3150800268413430360C4E70368202213430360C6E7C1
S315080026940368102213430360C8E703680822134338
S315080026A40360CAE70368042213430360CCE70133D3
S315080026B44268D20702D5064A9342F8D14368DB0733
S315080026C401D4012002E0002000E000207047C04643
S315080026D4FFFFFF0070B5837A01252A009A403D4B17
S315080026E48024A4001959294319518725AD0059593D
S315080026F4D44321405951037B002B18D1354D8321EE
S3150800270489006B5823406B50837AC188090446882C
S3150800271431434833DB005951837A81880904058893
S3150800272429434833DB002B4DAC4663445960037B8D
S31508002734012B1FD0C37A002B36D1264D812189005F
S315080027446B5823406B500389002B05D1214D8521F5
S3150800275489006B581C406C500389012B2BD0437B92
S31508002764012B2FD01B49802292008B5801208343CA
S315080027748B5070BD174D832189006B5813436B50DA
S31508002784837A01880904468831434833DB00595162
S31508002794837A81880904C58829434833DB000D4DAB
S315080027A4AC4663445960C5E70A4D812189006B58D4
S315080027B413436B50C7E7074C8521890063581343B5
S315080027C46350CCE7034987239B00C8580243CA5081
S315080027D4C8E7C0460064004000238371C3710372CE
S315080027E443728372C3728370C37003330371013BEC
S315080027F44371013B0380704730B50B001B331B0143
S315080028041C5804232340137238D10B001B331B01B5
S315080028141B585B0D13600B001B331B011D58022448
S315080028242C405472C3185D680F242C4094725B685C
S315080028341B0AD3740B01C3181C00B934FF3425686A
S31508002844D57225682D0A157325682D0C55732468C9
S31508002854240E9473BD33FF331C68D4731C68240A8E
S3150800286414741C68240C54741B681B0E9374002976
S315080028740BD0036920221343036130BD0B001B33BD
S315080028841B011B58DB085360C5E7C36820221343A2
S31508002894C360F2E7002903D0012905D0002002E02D
S315080028A4C068032318407047006903231840FAE7F1
S315080028B470B500222FE0836855000324AC40A34377
S315080028C4836083684C79AC4023438360838815040A
S315080028D42D0C0124AC40A343838086888C79AC40B4
S315080028E4A3B2334383800468550003231E00AE4015
S315080028F4B443046004680E79AE4034430460C46883
S315080029041604F60BB3409C43C460C368CC79AC4048
S315080029142343C36001320F2A0BD8012393400C6862
S315080029241C40A342F6D10B79013BDBB2012BDAD862
S31508002934C1E770BD816170470185704730B50723CB
S315080029440B409B009A40C908083189000C580F258A
S315080029549D40AC430C500B581A430A5030BD000036
S31508002964F8B50400744B58680C23184004284DD055
S3150800297407D908284ED00C2865D1704B236000204F
S3150800298403E000285FD16E4B23606B4A516809093E
S315080029940F230B406B4FFB5CDBB226683100D94032
S315080029A40B00616055682D0A07212940795CC9B274
S315080029B4CB40A360126BD20549D4634AE2605E4AEF
S315080029C4126B52064DD4614A22615B4A126BD206D7
S315080029D44BD45B4A6261584A126B920747D1A3618A
S315080029E4554A116BC022920211425BD1E361524AE5
S315080029F4116BC0221203114200D076E023624E4BBB
S31508002A041B6B1B0600D493E06062F8BD4C4B236035
S31508002A140020BAE7484B5D685A68C0235B02AD0CD0
S31508002A240F20054002351A4203D1494868432060FD
S31508002A34ABE7414BDB6A0F21194001314048FFF7E8
S31508002A4463FB6843F3E73E4B236000209DE73A4A5D
S31508002A545268520402D45A08E260B0E79A08E2605F
S31508002A64ADE7802212022261AFE76661B3E7324A14
S31508002A74116B03220A40012A0ED02F4A116B032236
S31508002A840A40022A0AD02C4A116B03220A40032A56
S31508002A94A6D12B4AA261A3E7A661A1E78022120266
S31508002AA4A2619DE7244A126BC02189020A4080214B
S31508002AB449028A4213D0204A126BC02189020A406D
S31508002AC4802189028A420CD01B4A126BC0218902D2
S31508002AD40A408A4200D08AE7194AE26187E7E66132
S31508002AE485E780221202E26181E7134B1B6BC02241
S31508002AF4120313408022D202934213D00E4B1B6B4F
S31508002B04C022120313408022120393420CD00A4BAC
S31508002B141B6BC02212031340934200D06FE7084B85
S31508002B2423626CE726626AE780231B02236266E750
S31508002B34024B636269E7C04600100240006CDC027F
S31508002B4400127A00C0000020809FD5001280000081
S31508002B5400093D00002904D1044A5369834353619B
S31508002B647047024A536918435061F9E70010024056
S31508002B74002904D1044AD3698343D3617047024ABE
S31508002B84D3691843D061F9E700100240002904D13B
S31508002B94044A1369834313617047024A1369184345
S31508002BA41061F9E700100240F0B58DB004000D007D
S31508002BB4036801229343036043682A4A13408A68D8
S31508002BC4134343600368284A13404A68C9680A439A
S31508002BD429690A43134303608368244A13406A69CC
S31508002BE41343836002A8FFF7BBFE214B9C4227D000
S31508002BF4204B9C4226D0204B9C4225D0049E236819
S31508002C041B0423D576002B68019319003000FFF7BF
S31508002C147BFA070001993000FFF7FCFA2B685B087A
S31508002C24994200D3013723681B0405D57B0807227C
S31508002C341A40124B1F401743BBB2A3810DB0F0BD17
S31508002C44089EDCE7099EDAE70A9ED8E72B68019313
S31508002C5419003000FFF758FA070001993000FFF70A
S31508002C64D9FADBE7FFCFFFFFF3E9FFFFFFFCFFFF1E
S31508002C74003801400044004000480040F0FF0000CE
S31508002C84002904D10368012293430360704703684B
S31508002C94012213430360F9E7808CC005C00D704711
S31508002CA4C369194201D1002070470120FCE70000DE
S31508002CB41122144B1A60144B5A685A605A685A609F
S31508002CC45A6812490A405A605968A02292030A436C
S31508002CD45A601968802252040A431A600A4B1B6810
S31508002CE49B01FBD5084B5A6803218A435A605A68E4
S31508002CF401390A435A60044B5A680C231340082BBB
S31508002D04F9D170470020024000100240FF7FC0FF3F
S31508002D1410B5124B1A6801210A431A605A681048FA
S31508002D2402405A601A680F4802401A601A680E4828
S31508002D3402401A605A680D4802405A60DA6A0F203F
S31508002D448243DA621A6B0A4802401A635A6B8A4348
S31508002D545A6300229A60FFF7ABFF10BD00100240C9
S31508002D640CB8FFF8FFFFF6FEFFFFFBFFFFFFC0FFEF
S31508002D74ACFEFFFF10B5FFF7D7FB00F03BF810BD1C
S31508002D8410B5FFF7F7FFFFF73FFBFFF7EBFBFFF77E
S31508002D94C5FBFAE70D488546002103E00C4B5B5852
S31508002DA4435004310B480C4B42189A42F6D30B4A4B
S31508002DB402E0002313600432094B9A42F9D3FFF761
S31508002DC4A7FF00F04BF8FFF7DBFFFEE700800020C3
S31508002DD4F02E0008C0000020D4000020D4000020F3
S31508002DE444010020FEE70000014B18607047C04606
S31508002DF44001002010B50E4B1868FA218900FFF728
S31508002E0483F901380B4B98420DD80B4A50600B488E
S31508002E14036A1B021B0AC02109060B43036200232B
S31508002E249360073313600020FFF7DEFF10BDC0462A
S31508002E34D0000020FFFFFF0010E000E000ED00E0F6
S31508002E44014B18687047C04640010020024A1368BF
S31508002E54013313607047C0464001002070B5002650
S31508002E640C4D0D4C641BA410A64209D1002600F093
S31508002E7419F80A4D0A4C641BA410A64205D170BD64
S31508002E84B300EB5898470136EEE7B300EB5898477A
S31508002E940136F2E7E82E0008E82E0008E82E0008B6
S31508002EA4EC2E0008F8B5C046F8BC08BC9E46704728
S31108002EB4F8B5C046F8BC08BC9E4670473E
S31508002EC001010000050206020603070308030903B9
S31508002ED009040A040B040C040C050D050E050F0560
S30D08002EE00F0610061007100882
S30908002EE8ED200008C3
S30908002EECC5200008E7
S31508002EF00000000001020304010203040607080992
S30908002F00006CDC0275
S70508002D992C
